:100000008CC0B0C0AFC0AEC0ADC0B1C0ABC0AAC0A4
:10001000A9C0A8C0A7C0A6C0A5C0A4C0A3C074455D
:1000200079467D47824887498B60906194629963E5
:100030009D64A265A766AB67B068B469B980BE81EC
:10004000C282C783CB84D084D484FF210000000007
:100050000000000000000000000023456C98C9FF6C
:10006000040714233764A0FFFFFFFFFFFFFFFFFF1C
:10007000FFFFFF00000000000000000023405F7A47
:10008000B4FFFFFFFFFFFF001400081400080E1468
:100090000004080E14000305080E140004080A0EDC
:1000A0001114000305080A0E1014000305080A0EB7
:1000B0001012140008000E00080E0004080E0003C1
:1000C00005080E0004080E1100080E1100F3F404D8
:1000D000080E10121400080A0C0E0F10121400085B
:1000E0000EED14000203040500041400040E1400B5
:1000F000040810140004080F1114000305080A0E68
:100100000004080A0E00EEEDECEB140E08040004E7
:10011000080E00EBECEDEEF3F41411241FBECFE556
:10012000D1E0DEBFCDBF20E0A0E6B0E001C01D926F
:10013000A937B207E1F7EAE7F0E085E5808781E0DB
:10014000838314821282868311828BE0818788E503
:100150008287E0E6F0E08DEF87838EEF8583712C58
:10016000B1D0B8C24DCF1BBC19BC18BC08951895AE
:1001700025B7277E25BF29B7226029BF21E022BFEE
:10018000019728F020E188952150E9F7F9CF0895EB
:1001900088EE93E0EDCF369A3699FECF85B108957B
:1001A000CF93C72D81E0870D8F73782E662D90E059
:1001B00083D26FEF8C2F90E0CF917EC2FF920F938E
:1001C0001F93CF93DF93F82E0BE710E0CEE7D0E03C
:1001D000F11005C0CE0168D2F801808304C0F80197
:1001E0006081CE0169D221970F5F1F4FC437D105BF
:1001F00079F7DF91CF911F910F91FF900895D0DF94
:1002000081E0DCCF811101C0AECF815090E0FC01D4
:10021000E45BFF4FE491EBBDFC01E05AFF4FE4913A
:10022000E9BDFC01EC58FF4F849188BD08950F9300
:100230001F93CF93C82F8B01CC2359F085E0E2DFC9
:10024000C80196DF90DFC80193DFC80191DFC1507C
:10025000F3CFCF911F910F910895EF92FF920F93DB
:100260001F93CF93C8E0E82EF12C062F10E084E115
:10027000C9DFC7017DDF77DFC8017ADFC150B9F779
:10028000CF911F910F91FF90EF9008951F93CF93FF
:10029000DF938FEA87B986EC86B910E1C0E0D0E041
:1002A00085E090E065DF77DFC80FD11D1150C1F701
:1002B000CE0124E0969587952A95E1F7DF91CF91BD
:1002C0001F9108951092790083EA87B986EC86B968
:1002D0003699FECF369A3699FECF85B18095582E45
:1002E00087E790E0E1D1853519F0612C88DF11C0F6
:1002F000712C872D90E0D8D1682E8F3F19F080E0C7
:100300005DDF07C0872D91E0970D792E803488F34B
:10031000F6CF20918300C0917D0010917E008091E6
:100320007B00882319F010E0C0E02AE12F5F90E005
:1003300040E050E0A8E8B0E0222379F0BD016F5F13
:100340007F4FFB013197E491EE2319F0962F9A1B12
:10035000F6CF2150AD01DB01EFCF092F6C2F70E0FC
:10036000A92FB0E0E02FF0E0112321F09D012E1B1A
:100370003F0B05C09F0121503109260F371F3197D0
:10038000E40FF51FF49027593F4FF901F082015017
:1003900049F79C0F90938500CC2371F0112329F02D
:1003A000292F30E02150310902C020E030E0F9016E
:1003B000E759FF4F41E0408327E0290F322F3150AA
:1003C000E32FE91BF0E0ED5EFE4FE491A32FB0E0D8
:1003D000A759BF4FEC933913F2CFE22FF0E0E85961
:1003E000FF4F31E0509169004081541330E0231BEE
:1003F00020938600362D353FE8F5452D4134B0F485
:10040000809187008F3F29F4809179008093870045
:1004100006C081E0860D682E891708F0612C809156
:1004200087008F5F8F718093870024C0309179009F
:10043000309387004F3AC0F430918000332311F09D
:10044000882339F081E0860D682E891798F0612C99
:1004500011C0862D6916D9F3662019F08150682ED7
:1004600009C02150622E06C08111F1CF80917C001D
:10047000882369F38FEF8DBD80E68CBD8FE384BB4D
:100480008BE187BB88EE88BB81E083BF91EA9ABD90
:1004900080BF85B7806285BF789497B986EC86B9AE
:1004A000C62DC53F10F0612C3CC080918700803183
:1004B00038F4E62DF0E0E759FF4FC081DC2F31C062
:1004C00067DE8091790080938700CBE7D0E000E081
:1004D00010E0FF24F39481E0800F0F5F1F4F98819D
:1004E0009F3F29F4219608301105A9F7E2CF6DE569
:1004F00070E09DDEF801E05AFF4F608088818F2513
:1005000088837DDE6FE070E080E291DE88818F2558
:100510008883612C74DE3CDE80917B00882311F39C
:10052000C8CF3EDE10E0F12C81EAE82E96ECD92E01
:10053000CC24CA94CE3E19F463E481E204C0CD3EDB
:1005400021F468E284E189DE6FC0CC3E11F469E2F7
:1005500003C0CB3E19F462E581E0F5CFC33F81F4DF
:1005600004E084E14FDE85E090E002DE88E04ADED0
:1005700081E490E0FDDD0150A1F780ED92E053C0F1
:10058000C43F51F584E690E0F3DD05DE90E0292FCD
:1005900030E0F901E25EFF4FE491E81710F49E5F4E
:1005A000F6CFF901E15EFF4F04916DE770E0802F17
:1005B0008295869587703BDE8EEE92E0D9DD65E010
:1005C00070E081E034DE85E694E0D2DD6DE770E036
:1005D000802F8F712CDE0DC0CE3F71F400E00093B0
:1005E00083000DDE6AEF70E081E021DE0F5F0A31EB
:1005F000B1F7CEDDCDDD18C0CD3F39F58FEF80935B
:100600008400FDDD85E0FEDDC3DDC2DD84E1FADDD1
:100610003DDE80938400F3DDBBDDBADDF9CFDB3056
:10062000F8F484EF91E0A4DD809179008093870055
:10063000B2DD823808F036C01F5F183008F47ACF78
:10064000D531A8F010E0DAE0CAE08D2FDBDD1EDE48
:10065000E7B8D6B8F39490918400891710F3DFCFF0
:10066000F4E1FF15F0F6C0927900DAE0DACFD2308B
:1006700030F08D2F86958695D695D80F12C073DDF4
:1006800085B7877E806185BFF89485B7846885BF0C
:100690008B7F85BF85B7806285BF889585B78F7D45
:1006A00085BFCD2F10E046CFE199FECF1FBA8EBB9C
:1006B000E09A99278DB30895262FE199FECF1CBAB1
:1006C0001FBA8EBB2DBB0FB6F894E29AE19A0FBE0B
:0806D00001960895F894FFCF94
